ARM Linker, 4.1 [Build 567] [Standard]

==============================================================================

Section Cross References

    startup_lpc11xx.o(RESET) refers to startup_lpc11xx.o(STACK) for __initial_sp
    startup_lpc11xx.o(RESET) refers to startup_lpc11xx.o(.text) for Reset_Handler
    startup_lpc11xx.o(RESET) refers to lpc11c14_it.o(.text) for NMI_Handler
    startup_lpc11xx.o(RESET) refers to os_cpu_a.o(.text) for OS_CPU_PendSVHandler
    startup_lpc11xx.o(RESET) refers to os_cpu_c.o(.text) for OS_CPU_SysTickHandler
    startup_lpc11xx.o(RESET) refers to ssp.o(.text) for SSP1_IRQHandler
    startup_lpc11xx.o(RESET) refers to i2c.o(.text) for I2C_IRQHandler
    startup_lpc11xx.o(RESET) refers to uart.o(.text) for UART_IRQHandler
    startup_lpc11xx.o(RESET) refers to gpio.o(.text) for PIOINT3_IRQHandler
    startup_lpc11xx.o(.text) refers to entry.o(.ARM.Collect$$$$00000000) for __main
    system_lpc11xx.o(.text) refers to system_lpc11xx.o(.data) for ClockSource
    gpio.o(.text) refers to os_time.o(.text) for OSTimeDlyResume
    gpio.o(.text) refers to spi_uart.o(.text) for ZigBee_IRQ_Process
    gpio.o(.text) refers to gpio.o(.data) for gpio0_counter
    gpio.o(.text) refers to gpio.o(.constdata) for LPC_GPIO
    uart.o(.text) refers to uidiv.o(.text) for __aeabi_uidivmod
    uart.o(.text) refers to printfa.o(i.__0vsnprintf) for __c89vsnprintf
    uart.o(.text) refers to uart.o(.data) for UARTStatus
    uart.o(.text) refers to uart.o(.bss) for UARTBuffer
    uart.o(.text) refers to system_lpc11xx.o(.data) for SystemAHBFrequency
    retarget.o(.text) refers to uart.o(.data) for UARTCount
    retarget.o(.text) refers to uart.o(.bss) for UARTBuffer
    i2c.o(.text) refers to i2c.o(i.__ARM_common_switch8) for __ARM_common_switch8
    i2c.o(.text) refers to i2c.o(.data) for WrIndex
    adc.o(.text) refers to uidiv.o(.text) for __aeabi_uidivmod
    adc.o(.text) refers to adc.o(.bss) for ADCValue
    adc.o(.text) refers to system_lpc11xx.o(.data) for SystemAHBFrequency
    ssp.o(.text) refers to gpio.o(.text) for GPIOSetDir
    ssp.o(.text) refers to ssp.o(.data) for interruptOverRunStat0
    tools.o(.text) refers to uidiv.o(.text) for __aeabi_uidivmod
    key.o(.text) refers to gpio.o(.text) for GPIOSetDir
    seg7led.o(.text) refers to gpio.o(.text) for GPIOSetDir
    seg7led.o(.text) refers to seg7led.o(.constdata) for segcode
    temp_hum.o(.text) refers to gpio.o(.text) for GPIOSetDir
    temp_hum.o(.text) refers to tools.o(.text) for delay_ms
    temp_hum.o(.text) refers to gpio.o(.data) for p3_2_counter
    light.o(.text) refers to i2c.o(.text) for I2CWrite
    light.o(.text) refers to uidiv.o(.text) for __aeabi_uidivmod
    light.o(.text) refers to gpio.o(.text) for GPIOIntDisable
    light.o(.text) refers to light.o(.data) for range
    acc.o(.text) refers to i2c.o(.text) for I2CWrite
    rfid.o(.text) refers to ssp.o(.text) for SPI_Init
    rfid.o(.text) refers to tools.o(.text) for delay_ms
    rfid.o(.text) refers to gpio.o(.text) for GPIOSetValue
    rfid.o(.text) refers to rfid.o(.constdata) for RFID_READ_CARD_20
    spi_uart.o(.text) refers to gpio.o(.text) for GPIOSetValue
    spi_uart.o(.text) refers to ssp.o(.text) for SPI_PutGet
    spi_uart.o(.text) refers to uart.o(.text) for UART0_PutChar
    spi_uart.o(.text) refers to uidiv.o(.text) for __aeabi_uidivmod
    spi_uart.o(.text) refers to spi_uart.o(.bss) for SPI752_rbuf_0
    spi_uart.o(.text) refers to spi_uart.o(.data) for SPI752_rbuf_0_ip
    os_cpu_a.o(.text) refers to os_core.o(.data) for OSRunning
    os_cpu_a.o(.text) refers to os_cpu_c.o(.text) for OSTaskSwHook
    os_cpu_c.o(.text) refers to os_cpu_a.o(.text) for OS_CPU_SR_Save
    os_cpu_c.o(.text) refers to os_core.o(.text) for OSTimeTick
    os_cpu_c.o(.text) refers to os_core.o(.data) for OSIntNesting
    os_core.o(.text) refers to os_cpu_a.o(.text) for OS_CPU_SR_Save
    os_core.o(.text) refers to i2c.o(i.__ARM_common_switch8) for __ARM_common_switch8
    os_core.o(.text) refers to os_core.o(.data) for OSIntNesting
    os_core.o(.text) refers to os_core.o(.constdata) for OSUnMapTbl
    os_core.o(.text) refers to os_core.o(.bss) for OSRdyTbl
    os_core.o(.text) refers to os_task.o(.text) for OSTaskStkChk
    os_core.o(.text) refers to os_time.o(.text) for OSTimeDly
    os_core.o(.text) refers to uidiv.o(.text) for __aeabi_uidivmod
    os_core.o(.text) refers to os_cpu_c.o(.text) for OSTaskStatHook
    os_core.o(.text) refers to os_flag.o(.text) for OS_FlagInit
    os_core.o(.text) refers to os_mem.o(.text) for OS_MemInit
    os_core.o(.text) refers to os_q.o(.text) for OS_QInit
    os_flag.o(.text) refers to os_cpu_a.o(.text) for OS_CPU_SR_Save
    os_flag.o(.text) refers to os_core.o(.text) for OS_Sched
    os_flag.o(.text) refers to os_core.o(.data) for OSIntNesting
    os_flag.o(.text) refers to os_core.o(.bss) for OSRdyTbl
    os_mbox.o(.text) refers to os_cpu_a.o(.text) for OS_CPU_SR_Save
    os_mbox.o(.text) refers to os_core.o(.text) for OS_EventWaitListInit
    os_mbox.o(.text) refers to os_core.o(.data) for OSIntNesting
    os_mem.o(.text) refers to os_cpu_a.o(.text) for OS_CPU_SR_Save
    os_mem.o(.text) refers to os_core.o(.text) for OS_StrLen
    os_mem.o(.text) refers to os_core.o(.data) for OSMemFreeList
    os_mem.o(.text) refers to os_core.o(.bss) for OSMemTbl
    os_mutex.o(.text) refers to os_cpu_a.o(.text) for OS_CPU_SR_Save
    os_mutex.o(.text) refers to os_core.o(.text) for OS_EventWaitListInit
    os_mutex.o(.text) refers to os_core.o(.data) for OSIntNesting
    os_mutex.o(.text) refers to os_core.o(.bss) for OSTCBPrioTbl
    os_q.o(.text) refers to os_cpu_a.o(.text) for OS_CPU_SR_Save
    os_q.o(.text) refers to os_core.o(.text) for OS_EventWaitListInit
    os_q.o(.text) refers to os_core.o(.data) for OSIntNesting
    os_q.o(.text) refers to os_core.o(.bss) for OSQTbl
    os_sem.o(.text) refers to os_cpu_a.o(.text) for OS_CPU_SR_Save
    os_sem.o(.text) refers to os_core.o(.text) for OS_EventWaitListInit
    os_sem.o(.text) refers to os_core.o(.data) for OSIntNesting
    os_task.o(.text) refers to os_cpu_a.o(.text) for OS_CPU_SR_Save
    os_task.o(.text) refers to os_core.o(.text) for OS_Sched
    os_task.o(.text) refers to os_cpu_c.o(.text) for OSTaskStkInit
    os_task.o(.text) refers to os_flag.o(.text) for OS_FlagUnlink
    os_task.o(.text) refers to os_core.o(.bss) for OSTCBPrioTbl
    os_task.o(.text) refers to os_core.o(.data) for OSTCBCur
    os_time.o(.text) refers to os_cpu_a.o(.text) for OS_CPU_SR_Save
    os_time.o(.text) refers to os_core.o(.text) for OS_Sched
    os_time.o(.text) refers to uidiv.o(.text) for __aeabi_uidivmod
    os_time.o(.text) refers to os_core.o(.data) for OSIntNesting
    os_time.o(.text) refers to os_core.o(.bss) for OSRdyTbl
    main.o(.text) refers to led_spk_fan_adc.o(.text) for send_package
    main.o(.text) refers to os_time.o(.text) for OSTimeDlyHMSM
    main.o(.text) refers to gpio.o(.text) for GPIOSetDir
    main.o(.text) refers to uart.o(.text) for UARTInit
    main.o(.text) refers to rfid.o(.text) for RFID_Collect
    main.o(.text) refers to acc.o(.text) for acc_init
    main.o(.text) refers to adc.o(.text) for ADCInit
    main.o(.text) refers to light.o(.text) for light_init
    main.o(.text) refers to temp_hum.o(.text) for Temp_Hum_Collect
    main.o(.text) refers to os_sem.o(.text) for OSSemPend
    main.o(.text) refers to printfb.o(i.__0printf$bare) for __2printf
    main.o(.text) refers to key.o(.text) for KEY_Read
    main.o(.text) refers to os_mbox.o(.text) for OSMboxPend
    main.o(.text) refers to uidiv.o(.text) for __aeabi_uidivmod
    main.o(.text) refers to seg7led.o(.text) for Seg7Led_Put
    main.o(.text) refers to os_cpu_c.o(.text) for OS_CPU_SysTickInit
    main.o(.text) refers to os_core.o(.text) for OSStatInit
    main.o(.text) refers to os_task.o(.text) for OSTaskDel
    main.o(.text) refers to system_lpc11xx.o(.text) for SystemInit
    main.o(.text) refers to ssp.o(.text) for SPI_IOConfig
    main.o(.text) refers to spi_uart.o(.text) for SPI752_Init
    main.o(.text) refers to i2c.o(.text) for I2CInit
    main.o(.text) refers to main.o(.data) for dev_info
    main.o(.text) refers to gpio.o(.data) for p2_8_counter
    main.o(.text) refers to main.o(.bss) for Task_Start_STK
    main.o(.data) refers to main.o(.bss) for dev
    lpc11c14_it.o(.text) refers to os_cpu_a.o(.text) for OS_CPU_PendSVHandler
    lpc11c14_it.o(.text) refers to os_cpu_c.o(.text) for OS_CPU_SysTickHandler
    crc16.o(.text) refers to crc16.o(.constdata) for crc16_table
    led_spk_fan_adc.o(.text) refers to adc.o(.text) for ADCRead
    led_spk_fan_adc.o(.text) refers to crc16.o(.text) for make_crc16
    led_spk_fan_adc.o(.text) refers to uart.o(.text) for UARTSend
    led_spk_fan_adc.o(.text) refers to spi_uart.o(.text) for ZigBee_Send
    entry.o(.ARM.Collect$$$$00000000) refers (Special) to entry7.o(.ARM.Collect$$$$00000007) for _main_init
    entry.o(.ARM.Collect$$$$00000000) refers (Special) to entry5.o(.ARM.Collect$$$$00000004) for _main_scatterload
    entry.o(.ARM.Collect$$$$00000000) refers (Special) to entry2.o(.ARM.Collect$$$$00000001) for _main_stk
    printfb.o(i.__0fprintf$bare) refers to printfb.o(i._printf_core) for _printf_core
    printfb.o(i.__0fprintf$bare) refers to retarget.o(.text) for fputc
    printfb.o(i.__0printf$bare) refers to printfb.o(i._printf_core) for _printf_core
    printfb.o(i.__0printf$bare) refers to retarget.o(.text) for fputc
    printfb.o(i.__0printf$bare) refers to retarget.o(.data) for __stdout
    printfb.o(i.__0snprintf$bare) refers to printfb.o(i._printf_core) for _printf_core
    printfb.o(i.__0snprintf$bare) refers to printfb.o(i._snputc) for _snputc
    printfb.o(i.__0sprintf$bare) refers to printfb.o(i._printf_core) for _printf_core
    printfb.o(i.__0sprintf$bare) refers to printfb.o(i._sputc) for _sputc
    printfb.o(i.__0vfprintf$bare) refers to printfb.o(i._printf_core) for _printf_core
    printfb.o(i.__0vfprintf$bare) refers to retarget.o(.text) for fputc
    printfb.o(i.__0vprintf$bare) refers to printfb.o(i._printf_core) for _printf_core
    printfb.o(i.__0vprintf$bare) refers to retarget.o(.text) for fputc
    printfb.o(i.__0vprintf$bare) refers to retarget.o(.data) for __stdout
    printfb.o(i.__0vsnprintf$bare) refers to printfb.o(i._printf_core) for _printf_core
    printfb.o(i.__0vsnprintf$bare) refers to printfb.o(i._snputc) for _snputc
    printfb.o(i.__0vsprintf$bare) refers to printfb.o(i._printf_core) for _printf_core
    printfb.o(i.__0vsprintf$bare) refers to printfb.o(i._sputc) for _sputc
    printf0.o(i.__0fprintf$0) refers to printf0.o(i._printf_core) for _printf_core
    printf0.o(i.__0fprintf$0) refers to retarget.o(.text) for fputc
    printf0.o(i.__0printf$0) refers to printf0.o(i._printf_core) for _printf_core
    printf0.o(i.__0printf$0) refers to retarget.o(.text) for fputc
    printf0.o(i.__0printf$0) refers to retarget.o(.data) for __stdout
    printf0.o(i.__0snprintf$0) refers to printf0.o(i._printf_core) for _printf_core
    printf0.o(i.__0snprintf$0) refers to printf0.o(i._snputc) for _snputc
    printf0.o(i.__0sprintf$0) refers to printf0.o(i._printf_core) for _printf_core
    printf0.o(i.__0sprintf$0) refers to printf0.o(i._sputc) for _sputc
    printf0.o(i.__0vfprintf$0) refers to printf0.o(i._printf_core) for _printf_core
    printf0.o(i.__0vfprintf$0) refers to retarget.o(.text) for fputc
    printf0.o(i.__0vprintf$0) refers to printf0.o(i._printf_core) for _printf_core
    printf0.o(i.__0vprintf$0) refers to retarget.o(.text) for fputc
    printf0.o(i.__0vprintf$0) refers to retarget.o(.data) for __stdout
    printf0.o(i.__0vsnprintf$0) refers to printf0.o(i._printf_core) for _printf_core
    printf0.o(i.__0vsnprintf$0) refers to printf0.o(i._snputc) for _snputc
    printf0.o(i.__0vsprintf$0) refers to printf0.o(i._printf_core) for _printf_core
    printf0.o(i.__0vsprintf$0) refers to printf0.o(i._sputc) for _sputc
    printf1.o(i.__0fprintf$1) refers to printf1.o(i._printf_core) for _printf_core
    printf1.o(i.__0fprintf$1) refers to retarget.o(.text) for fputc
    printf1.o(i.__0printf$1) refers to printf1.o(i._printf_core) for _printf_core
    printf1.o(i.__0printf$1) refers to retarget.o(.text) for fputc
    printf1.o(i.__0printf$1) refers to retarget.o(.data) for __stdout
    printf1.o(i.__0snprintf$1) refers to printf1.o(i._printf_core) for _printf_core
    printf1.o(i.__0snprintf$1) refers to printf1.o(i._snputc) for _snputc
    printf1.o(i.__0sprintf$1) refers to printf1.o(i._printf_core) for _printf_core
    printf1.o(i.__0sprintf$1) refers to printf1.o(i._sputc) for _sputc
    printf1.o(i.__0vfprintf$1) refers to printf1.o(i._printf_core) for _printf_core
    printf1.o(i.__0vfprintf$1) refers to retarget.o(.text) for fputc
    printf1.o(i.__0vprintf$1) refers to printf1.o(i._printf_core) for _printf_core
    printf1.o(i.__0vprintf$1) refers to retarget.o(.text) for fputc
    printf1.o(i.__0vprintf$1) refers to retarget.o(.data) for __stdout
    printf1.o(i.__0vsnprintf$1) refers to printf1.o(i._printf_core) for _printf_core
    printf1.o(i.__0vsnprintf$1) refers to printf1.o(i._snputc) for _snputc
    printf1.o(i.__0vsprintf$1) refers to printf1.o(i._printf_core) for _printf_core
    printf1.o(i.__0vsprintf$1) refers to printf1.o(i._sputc) for _sputc
    printf1.o(i._printf_core) refers to uidiv.o(.text) for __aeabi_uidivmod
    printf2.o(i.__0fprintf$2) refers to printf2.o(i._printf_core) for _printf_core
    printf2.o(i.__0fprintf$2) refers to retarget.o(.text) for fputc
    printf2.o(i.__0printf$2) refers to printf2.o(i._printf_core) for _printf_core
    printf2.o(i.__0printf$2) refers to retarget.o(.text) for fputc
    printf2.o(i.__0printf$2) refers to retarget.o(.data) for __stdout
    printf2.o(i.__0snprintf$2) refers to printf2.o(i._printf_core) for _printf_core
    printf2.o(i.__0snprintf$2) refers to printf2.o(i._snputc) for _snputc
    printf2.o(i.__0sprintf$2) refers to printf2.o(i._printf_core) for _printf_core
    printf2.o(i.__0sprintf$2) refers to printf2.o(i._sputc) for _sputc
    printf2.o(i.__0vfprintf$2) refers to printf2.o(i._printf_core) for _printf_core
    printf2.o(i.__0vfprintf$2) refers to retarget.o(.text) for fputc
    printf2.o(i.__0vprintf$2) refers to printf2.o(i._printf_core) for _printf_core
    printf2.o(i.__0vprintf$2) refers to retarget.o(.text) for fputc
    printf2.o(i.__0vprintf$2) refers to retarget.o(.data) for __stdout
    printf2.o(i.__0vsnprintf$2) refers to printf2.o(i._printf_core) for _printf_core
    printf2.o(i.__0vsnprintf$2) refers to printf2.o(i._snputc) for _snputc
    printf2.o(i.__0vsprintf$2) refers to printf2.o(i._printf_core) for _printf_core
    printf2.o(i.__0vsprintf$2) refers to printf2.o(i._sputc) for _sputc
    printf3.o(i.__0fprintf$3) refers to printf3.o(i._printf_core) for _printf_core
    printf3.o(i.__0fprintf$3) refers to retarget.o(.text) for fputc
    printf3.o(i.__0printf$3) refers to printf3.o(i._printf_core) for _printf_core
    printf3.o(i.__0printf$3) refers to retarget.o(.text) for fputc
    printf3.o(i.__0printf$3) refers to retarget.o(.data) for __stdout
    printf3.o(i.__0snprintf$3) refers to printf3.o(i._printf_core) for _printf_core
    printf3.o(i.__0snprintf$3) refers to printf3.o(i._snputc) for _snputc
    printf3.o(i.__0sprintf$3) refers to printf3.o(i._printf_core) for _printf_core
    printf3.o(i.__0sprintf$3) refers to printf3.o(i._sputc) for _sputc
    printf3.o(i.__0vfprintf$3) refers to printf3.o(i._printf_core) for _printf_core
    printf3.o(i.__0vfprintf$3) refers to retarget.o(.text) for fputc
    printf3.o(i.__0vprintf$3) refers to printf3.o(i._printf_core) for _printf_core
    printf3.o(i.__0vprintf$3) refers to retarget.o(.text) for fputc
    printf3.o(i.__0vprintf$3) refers to retarget.o(.data) for __stdout
    printf3.o(i.__0vsnprintf$3) refers to printf3.o(i._printf_core) for _printf_core
    printf3.o(i.__0vsnprintf$3) refers to printf3.o(i._snputc) for _snputc
    printf3.o(i.__0vsprintf$3) refers to printf3.o(i._printf_core) for _printf_core
    printf3.o(i.__0vsprintf$3) refers to printf3.o(i._sputc) for _sputc
    printf3.o(i._printf_core) refers to uidiv.o(.text) for __aeabi_uidivmod
    printf4.o(i.__0fprintf$4) refers to printf4.o(i._printf_core) for _printf_core
    printf4.o(i.__0fprintf$4) refers to retarget.o(.text) for fputc
    printf4.o(i.__0printf$4) refers to printf4.o(i._printf_core) for _printf_core
    printf4.o(i.__0printf$4) refers to retarget.o(.text) for fputc
    printf4.o(i.__0printf$4) refers to retarget.o(.data) for __stdout
    printf4.o(i.__0snprintf$4) refers to printf4.o(i._printf_core) for _printf_core
    printf4.o(i.__0snprintf$4) refers to printf4.o(i._snputc) for _snputc
    printf4.o(i.__0sprintf$4) refers to printf4.o(i._printf_core) for _printf_core
    printf4.o(i.__0sprintf$4) refers to printf4.o(i._sputc) for _sputc
    printf4.o(i.__0vfprintf$4) refers to printf4.o(i._printf_core) for _printf_core
    printf4.o(i.__0vfprintf$4) refers to retarget.o(.text) for fputc
    printf4.o(i.__0vprintf$4) refers to printf4.o(i._printf_core) for _printf_core
    printf4.o(i.__0vprintf$4) refers to retarget.o(.text) for fputc
    printf4.o(i.__0vprintf$4) refers to retarget.o(.data) for __stdout
    printf4.o(i.__0vsnprintf$4) refers to printf4.o(i._printf_core) for _printf_core
    printf4.o(i.__0vsnprintf$4) refers to printf4.o(i._snputc) for _snputc
    printf4.o(i.__0vsprintf$4) refers to printf4.o(i._printf_core) for _printf_core
    printf4.o(i.__0vsprintf$4) refers to printf4.o(i._sputc) for _sputc
    printf4.o(i._printf_core) refers to uldiv.o(.text) for __aeabi_uldivmod
    printf5.o(i.__0fprintf$5) refers to printf5.o(i._printf_core) for _printf_core
    printf5.o(i.__0fprintf$5) refers to retarget.o(.text) for fputc
    printf5.o(i.__0printf$5) refers to printf5.o(i._printf_core) for _printf_core
    printf5.o(i.__0printf$5) refers to retarget.o(.text) for fputc
    printf5.o(i.__0printf$5) refers to retarget.o(.data) for __stdout
    printf5.o(i.__0snprintf$5) refers to printf5.o(i._printf_core) for _printf_core
    printf5.o(i.__0snprintf$5) refers to printf5.o(i._snputc) for _snputc
    printf5.o(i.__0sprintf$5) refers to printf5.o(i._printf_core) for _printf_core
    printf5.o(i.__0sprintf$5) refers to printf5.o(i._sputc) for _sputc
    printf5.o(i.__0vfprintf$5) refers to printf5.o(i._printf_core) for _printf_core
    printf5.o(i.__0vfprintf$5) refers to retarget.o(.text) for fputc
    printf5.o(i.__0vprintf$5) refers to printf5.o(i._printf_core) for _printf_core
    printf5.o(i.__0vprintf$5) refers to retarget.o(.text) for fputc
    printf5.o(i.__0vprintf$5) refers to retarget.o(.data) for __stdout
    printf5.o(i.__0vsnprintf$5) refers to printf5.o(i._printf_core) for _printf_core
    printf5.o(i.__0vsnprintf$5) refers to printf5.o(i._snputc) for _snputc
    printf5.o(i.__0vsprintf$5) refers to printf5.o(i._printf_core) for _printf_core
    printf5.o(i.__0vsprintf$5) refers to printf5.o(i._sputc) for _sputc
    printf5.o(i._printf_core) refers to uldiv.o(.text) for __aeabi_uldivmod
    printf6.o(i.__0fprintf$6) refers to printf6.o(i._printf_core) for _printf_core
    printf6.o(i.__0fprintf$6) refers to retarget.o(.text) for fputc
    printf6.o(i.__0printf$6) refers to printf6.o(i._printf_core) for _printf_core
    printf6.o(i.__0printf$6) refers to retarget.o(.text) for fputc
    printf6.o(i.__0printf$6) refers to retarget.o(.data) for __stdout
    printf6.o(i.__0snprintf$6) refers to printf6.o(i._printf_core) for _printf_core
    printf6.o(i.__0snprintf$6) refers to printf6.o(i._snputc) for _snputc
    printf6.o(i.__0sprintf$6) refers to printf6.o(i._printf_core) for _printf_core
    printf6.o(i.__0sprintf$6) refers to printf6.o(i._sputc) for _sputc
    printf6.o(i.__0vfprintf$6) refers to printf6.o(i._printf_core) for _printf_core
    printf6.o(i.__0vfprintf$6) refers to retarget.o(.text) for fputc
    printf6.o(i.__0vprintf$6) refers to printf6.o(i._printf_core) for _printf_core
    printf6.o(i.__0vprintf$6) refers to retarget.o(.text) for fputc
    printf6.o(i.__0vprintf$6) refers to retarget.o(.data) for __stdout
    printf6.o(i.__0vsnprintf$6) refers to printf6.o(i._printf_core) for _printf_core
    printf6.o(i.__0vsnprintf$6) refers to printf6.o(i._snputc) for _snputc
    printf6.o(i.__0vsprintf$6) refers to printf6.o(i._printf_core) for _printf_core
    printf6.o(i.__0vsprintf$6) refers to printf6.o(i._sputc) for _sputc
    printf6.o(i._printf_core) refers to printf6.o(i._printf_pre_padding) for _printf_pre_padding
    printf6.o(i._printf_core) refers to printf6.o(i._printf_post_padding) for _printf_post_padding
    printf6.o(i._printf_core) refers to uidiv.o(.text) for __aeabi_uidivmod
    printf7.o(i.__0fprintf$7) refers to printf7.o(i._printf_core) for _printf_core
    printf7.o(i.__0fprintf$7) refers to retarget.o(.text) for fputc
    printf7.o(i.__0printf$7) refers to printf7.o(i._printf_core) for _printf_core
    printf7.o(i.__0printf$7) refers to retarget.o(.text) for fputc
    printf7.o(i.__0printf$7) refers to retarget.o(.data) for __stdout
    printf7.o(i.__0snprintf$7) refers to printf7.o(i._printf_core) for _printf_core
    printf7.o(i.__0snprintf$7) refers to printf7.o(i._snputc) for _snputc
    printf7.o(i.__0sprintf$7) refers to printf7.o(i._printf_core) for _printf_core
    printf7.o(i.__0sprintf$7) refers to printf7.o(i._sputc) for _sputc
    printf7.o(i.__0vfprintf$7) refers to printf7.o(i._printf_core) for _printf_core
    printf7.o(i.__0vfprintf$7) refers to retarget.o(.text) for fputc
    printf7.o(i.__0vprintf$7) refers to printf7.o(i._printf_core) for _printf_core
    printf7.o(i.__0vprintf$7) refers to retarget.o(.text) for fputc
    printf7.o(i.__0vprintf$7) refers to retarget.o(.data) for __stdout
    printf7.o(i.__0vsnprintf$7) refers to printf7.o(i._printf_core) for _printf_core
    printf7.o(i.__0vsnprintf$7) refers to printf7.o(i._snputc) for _snputc
    printf7.o(i.__0vsprintf$7) refers to printf7.o(i._printf_core) for _printf_core
    printf7.o(i.__0vsprintf$7) refers to printf7.o(i._sputc) for _sputc
    printf7.o(i._printf_core) refers to printf7.o(i._printf_pre_padding) for _printf_pre_padding
    printf7.o(i._printf_core) refers to printf7.o(i._printf_post_padding) for _printf_post_padding
    printf7.o(i._printf_core) refers to uldiv.o(.text) for __aeabi_uldivmod
    printf8.o(i.__0fprintf$8) refers to printf8.o(i._printf_core) for _printf_core
    printf8.o(i.__0fprintf$8) refers to retarget.o(.text) for fputc
    printf8.o(i.__0printf$8) refers to printf8.o(i._printf_core) for _printf_core
    printf8.o(i.__0printf$8) refers to retarget.o(.text) for fputc
    printf8.o(i.__0printf$8) refers to retarget.o(.data) for __stdout
    printf8.o(i.__0snprintf$8) refers to printf8.o(i._printf_core) for _printf_core
    printf8.o(i.__0snprintf$8) refers to printf8.o(i._snputc) for _snputc
    printf8.o(i.__0sprintf$8) refers to printf8.o(i._printf_core) for _printf_core
    printf8.o(i.__0sprintf$8) refers to printf8.o(i._sputc) for _sputc
    printf8.o(i.__0vfprintf$8) refers to printf8.o(i._printf_core) for _printf_core
    printf8.o(i.__0vfprintf$8) refers to retarget.o(.text) for fputc
    printf8.o(i.__0vprintf$8) refers to printf8.o(i._printf_core) for _printf_core
    printf8.o(i.__0vprintf$8) refers to retarget.o(.text) for fputc
    printf8.o(i.__0vprintf$8) refers to retarget.o(.data) for __stdout
    printf8.o(i.__0vsnprintf$8) refers to printf8.o(i._printf_core) for _printf_core
    printf8.o(i.__0vsnprintf$8) refers to printf8.o(i._snputc) for _snputc
    printf8.o(i.__0vsprintf$8) refers to printf8.o(i._printf_core) for _printf_core
    printf8.o(i.__0vsprintf$8) refers to printf8.o(i._sputc) for _sputc
    printf8.o(i._printf_core) refers to printf8.o(i._printf_pre_padding) for _printf_pre_padding
    printf8.o(i._printf_core) refers to printf8.o(i._printf_post_padding) for _printf_post_padding
    printf8.o(i._printf_core) refers to uldiv.o(.text) for __aeabi_uldivmod
    printfa.o(i.__0fprintf) refers (Special) to iusefp.o(.text) for __I$use$fp
    printfa.o(i.__0fprintf) refers to printfa.o(i._printf_core) for _printf_core
    printfa.o(i.__0fprintf) refers to retarget.o(.text) for fputc
    printfa.o(i.__0printf) refers (Special) to iusefp.o(.text) for __I$use$fp
    printfa.o(i.__0printf) refers to printfa.o(i._printf_core) for _printf_core
    printfa.o(i.__0printf) refers to retarget.o(.text) for fputc
    printfa.o(i.__0printf) refers to retarget.o(.data) for __stdout
    printfa.o(i.__0snprintf) refers (Special) to iusefp.o(.text) for __I$use$fp
    printfa.o(i.__0snprintf) refers to printfa.o(i._printf_core) for _printf_core
    printfa.o(i.__0snprintf) refers to printfa.o(i._snputc) for _snputc
    printfa.o(i.__0sprintf) refers (Special) to iusefp.o(.text) for __I$use$fp
    printfa.o(i.__0sprintf) refers to printfa.o(i._printf_core) for _printf_core
    printfa.o(i.__0sprintf) refers to printfa.o(i._sputc) for _sputc
    printfa.o(i.__0vfprintf) refers (Special) to iusefp.o(.text) for __I$use$fp
    printfa.o(i.__0vfprintf) refers to printfa.o(i._printf_core) for _printf_core
    printfa.o(i.__0vfprintf) refers to retarget.o(.text) for fputc
    printfa.o(i.__0vprintf) refers (Special) to iusefp.o(.text) for __I$use$fp
    printfa.o(i.__0vprintf) refers to printfa.o(i._printf_core) for _printf_core
    printfa.o(i.__0vprintf) refers to retarget.o(.text) for fputc
    printfa.o(i.__0vprintf) refers to retarget.o(.data) for __stdout
    printfa.o(i.__0vsnprintf) refers (Special) to iusefp.o(.text) for __I$use$fp
    printfa.o(i.__0vsnprintf) refers to printfa.o(i._printf_core) for _printf_core
    printfa.o(i.__0vsnprintf) refers to printfa.o(i._snputc) for _snputc
    printfa.o(i.__0vsprintf) refers (Special) to iusefp.o(.text) for __I$use$fp
    printfa.o(i.__0vsprintf) refers to printfa.o(i._printf_core) for _printf_core
    printfa.o(i.__0vsprintf) refers to printfa.o(i._sputc) for _sputc
    printfa.o(i._fp_digits) refers (Special) to iusefp.o(.text) for __I$use$fp
    printfa.o(i._fp_digits) refers to dmul.o(.text) for __aeabi_dmul
    printfa.o(i._fp_digits) refers to ddiv.o(.text) for __aeabi_ddiv
    printfa.o(i._fp_digits) refers to cdrcmple.o(.text) for __aeabi_cdrcmple
    printfa.o(i._fp_digits) refers to dadd.o(.text) for __aeabi_dadd
    printfa.o(i._fp_digits) refers to dfixul.o(.text) for __aeabi_d2ulz
    printfa.o(i._fp_digits) refers to uldiv.o(.text) for __aeabi_uldivmod
    printfa.o(i._printf_core) refers (Special) to iusefp.o(.text) for __I$use$fp
    printfa.o(i._printf_core) refers to printfa.o(i._printf_pre_padding) for _printf_pre_padding
    printfa.o(i._printf_core) refers to printfa.o(i._printf_post_padding) for _printf_post_padding
    printfa.o(i._printf_core) refers to uldiv.o(.text) for __aeabi_uldivmod
    printfa.o(i._printf_core) refers to printfa.o(i._fp_digits) for _fp_digits
    printfa.o(i._printf_core) refers to uidiv.o(.text) for __aeabi_uidivmod
    printfa.o(i._printf_post_padding) refers (Special) to iusefp.o(.text) for __I$use$fp
    printfa.o(i._printf_pre_padding) refers (Special) to iusefp.o(.text) for __I$use$fp
    printfa.o(i._snputc) refers (Special) to iusefp.o(.text) for __I$use$fp
    printfa.o(i._sputc) refers (Special) to iusefp.o(.text) for __I$use$fp
    entry2.o(.ARM.Collect$$$$00000001) refers to entry2.o(.ARM.Collect$$$$00002712) for __lit__00000000
    entry2.o(.ARM.Collect$$$$00002712) refers to startup_lpc11xx.o(STACK) for __initial_sp
    entry2.o(__vectab_stack_and_reset_area) refers to startup_lpc11xx.o(STACK) for __initial_sp
    entry2.o(__vectab_stack_and_reset_area) refers to entry.o(.ARM.Collect$$$$00000000) for __main
    entry5.o(.ARM.Collect$$$$00000004) refers to init.o(.text) for __scatterload
    entry7.o(.ARM.Collect$$$$00000007) refers to main.o(.text) for main
    uldiv.o(.text) refers to llushr.o(.text) for __aeabi_llsr
    uldiv.o(.text) refers to llshl.o(.text) for __aeabi_llsl
    dadd.o(.text) refers to llshl.o(.text) for __aeabi_llsl
    dadd.o(.text) refers to llsshr.o(.text) for __aeabi_lasr
    dadd.o(.text) refers to depilogue.o(.text) for _double_epilogue
    dmul.o(.text) refers to depilogue.o(.text) for _double_epilogue
    ddiv.o(.text) refers to depilogue.o(.text) for _double_round
    dfixul.o(.text) refers to llushr.o(.text) for __aeabi_llsr
    dfixul.o(.text) refers to llshl.o(.text) for __aeabi_llsl
    init.o(.text) refers to entry5.o(.ARM.Collect$$$$00000004) for __main_after_scatterload
    depilogue.o(.text) refers to depilogue.o(i.__ARM_clz) for __ARM_clz
    depilogue.o(.text) refers to llshl.o(.text) for __aeabi_llsl
    depilogue.o(.text) refers to llushr.o(.text) for __aeabi_llsr


==============================================================================

Removing Unused input sections from the image.

    Removing startup_lpc11xx.o(HEAP), (0 bytes).
    Removing core_cm0.o(.emb_text), (32 bytes).
    Removing adc.o(.data), (8 bytes).
    Removing ssp.o(.bss), (32 bytes).
    Removing ssp.o(.constdata), (16 bytes).
    Removing tools.o(.constdata), (16 bytes).
    Removing key.o(.constdata), (16 bytes).
    Removing temp_hum.o(.constdata), (16 bytes).
    Removing light.o(.constdata), (16 bytes).
    Removing spi_uart.o(.constdata), (16 bytes).
    Removing os_dbg.o(.constdata), (2 bytes).
    Removing os_mutex.o(.text), (1660 bytes).
    Removing main.o(.constdata), (17 bytes).
    Removing led_spk_fan_adc.o(.constdata), (16 bytes).

14 unused section(s) (total 1863 bytes) removed from the image.

==============================================================================

Image Symbol Table

    Local Symbols

    Symbol Name                              Value     Ov Type        Size  Object(Section)

    RESET                                    0x00000000   Section      192  startup_lpc11xx.o(RESET)
    ../../microlib/division.c                0x00000000   Number         0  uidiv.o ABSOLUTE
    ../../microlib/division.c                0x00000000   Number         0  uldiv.o ABSOLUTE
    ../../microlib/fpadd.c                   0x00000000   Number         0  dadd.o ABSOLUTE
    ../../microlib/fpdiv.c                   0x00000000   Number         0  ddiv.o ABSOLUTE
    ../../microlib/fpepilogue.c              0x00000000   Number         0  depilogue.o ABSOLUTE
    ../../microlib/fpfix.c                   0x00000000   Number         0  dfixul.o ABSOLUTE
    ../../microlib/fpmul.c                   0x00000000   Number         0  dmul.o ABSOLUTE
    ../../microlib/init/entry.s              0x00000000   Number         0  entry5.o ABSOLUTE
    ../../microlib/init/entry.s              0x00000000   Number         0  entry7.o ABSOLUTE
    ../../microlib/init/entry.s              0x00000000   Number         0  entry2.o ABSOLUTE
    ../../microlib/init/entry.s              0x00000000   Number         0  entry.o ABSOLUTE
    ../../microlib/longlong.c                0x00000000   Number         0  llushr.o ABSOLUTE
    ../../microlib/longlong.c                0x00000000   Number         0  llsshr.o ABSOLUTE
    ../../microlib/longlong.c                0x00000000   Number         0  llshl.o ABSOLUTE
    ../../microlib/printf/printf.c           0x00000000   Number         0  printf4.o ABSOLUTE
    ../../microlib/printf/printf.c           0x00000000   Number         0  printf8.o ABSOLUTE
    ../../microlib/printf/printf.c           0x00000000   Number         0  printf0.o ABSOLUTE
    ../../microlib/printf/printf.c           0x00000000   Number         0  printf1.o ABSOLUTE
    ../../microlib/printf/printf.c           0x00000000   Number         0  printf2.o ABSOLUTE
    ../../microlib/printf/printf.c           0x00000000   Number         0  printfa.o ABSOLUTE
    ../../microlib/printf/printf.c           0x00000000   Number         0  printf3.o ABSOLUTE
    ../../microlib/printf/printf.c           0x00000000   Number         0  printf7.o ABSOLUTE
    ../../microlib/printf/printf.c           0x00000000   Number         0  printf6.o ABSOLUTE
    ../../microlib/printf/printf.c           0x00000000   Number         0  printf5.o ABSOLUTE
    ../../microlib/printf/printf.c           0x00000000   Number         0  printfb.o ABSOLUTE
    ../../microlib/stubs.s                   0x00000000   Number         0  iusefp.o ABSOLUTE
    ../../microlib/stubs.s                   0x00000000   Number         0  useno.o ABSOLUTE
    ..\Lib_BSP\src\acc.c                     0x00000000   Number         0  acc.o ABSOLUTE
    ..\Lib_BSP\src\key.c                     0x00000000   Number         0  key.o ABSOLUTE
    ..\Lib_BSP\src\light.c                   0x00000000   Number         0  light.o ABSOLUTE
    ..\Lib_BSP\src\rfid.c                    0x00000000   Number         0  rfid.o ABSOLUTE
    ..\Lib_BSP\src\seg7led.c                 0x00000000   Number         0  seg7led.o ABSOLUTE
    ..\Lib_BSP\src\spi_uart.c                0x00000000   Number         0  spi_uart.o ABSOLUTE
    ..\Lib_BSP\src\temp_hum.c                0x00000000   Number         0  temp_hum.o ABSOLUTE
    ..\Lib_BSP\src\tools.c                   0x00000000   Number         0  tools.o ABSOLUTE
    ..\Lib_MCU\src\adc.c                     0x00000000   Number         0  adc.o ABSOLUTE
    ..\Lib_MCU\src\core_cm0.c                0x00000000   Number         0  core_cm0.o ABSOLUTE
    ..\Lib_MCU\src\gpio.c                    0x00000000   Number         0  gpio.o ABSOLUTE
    ..\Lib_MCU\src\i2c.c                     0x00000000   Number         0  i2c.o ABSOLUTE
    ..\Lib_MCU\src\retarget.c                0x00000000   Number         0  retarget.o ABSOLUTE
    ..\Lib_MCU\src\ssp.c                     0x00000000   Number         0  ssp.o ABSOLUTE
    ..\Lib_MCU\src\startup_LPC11xx.s         0x00000000   Number         0  startup_lpc11xx.o ABSOLUTE
    ..\Lib_MCU\src\system_LPC11xx.c          0x00000000   Number         0  system_lpc11xx.o ABSOLUTE
    ..\Lib_MCU\src\uart.c                    0x00000000   Number         0  uart.o ABSOLUTE
    ..\\Lib_MCU\\src\\core_cm0.c             0x00000000   Number         0  core_cm0.o ABSOLUTE
    ..\uCOS-II_V291\CPU\os_cpu_a.s           0x00000000   Number         0  os_cpu_a.o ABSOLUTE
    ..\uCOS-II_V291\CPU\os_cpu_c.c           0x00000000   Number         0  os_cpu_c.o ABSOLUTE
    ..\uCOS-II_V291\Source\os_core.c         0x00000000   Number         0  os_core.o ABSOLUTE
    ..\uCOS-II_V291\Source\os_dbg.c          0x00000000   Number         0  os_dbg.o ABSOLUTE
    ..\uCOS-II_V291\Source\os_flag.c         0x00000000   Number         0  os_flag.o ABSOLUTE
    ..\uCOS-II_V291\Source\os_mbox.c         0x00000000   Number         0  os_mbox.o ABSOLUTE
    ..\uCOS-II_V291\Source\os_mem.c          0x00000000   Number         0  os_mem.o ABSOLUTE
    ..\uCOS-II_V291\Source\os_mutex.c        0x00000000   Number         0  os_mutex.o ABSOLUTE
    ..\uCOS-II_V291\Source\os_q.c            0x00000000   Number         0  os_q.o ABSOLUTE
    ..\uCOS-II_V291\Source\os_sem.c          0x00000000   Number         0  os_sem.o ABSOLUTE
    ..\uCOS-II_V291\Source\os_task.c         0x00000000   Number         0  os_task.o ABSOLUTE
    ..\uCOS-II_V291\Source\os_time.c         0x00000000   Number         0  os_time.o ABSOLUTE
    ..\uCOS-II_V291\Source\os_tmr.c          0x00000000   Number         0  os_tmr.o ABSOLUTE
    cdrcmple.s                               0x00000000   Number         0  cdrcmple.o ABSOLUTE
    dc.s                                     0x00000000   Number         0  dc.o ABSOLUTE
    handlers.s                               0x00000000   Number         0  handlers.o ABSOLUTE
    init.s                                   0x00000000   Number         0  init.o ABSOLUTE
    src\crc16.c                              0x00000000   Number         0  crc16.o ABSOLUTE
    src\led_spk_fan_adc.c                    0x00000000   Number         0  led_spk_fan_adc.o ABSOLUTE
    src\lpc11c14_it.c                        0x00000000   Number         0  lpc11c14_it.o ABSOLUTE
    src\main.c                               0x00000000   Number         0  main.o ABSOLUTE
    .ARM.Collect$$$$00000000                 0x000000c0   Section        0  entry.o(.ARM.Collect$$$$00000000)
    .ARM.Collect$$$$00000001                 0x000000c0   Section        4  entry2.o(.ARM.Collect$$$$00000001)
    .ARM.Collect$$$$00000004                 0x000000c4   Section        4  entry5.o(.ARM.Collect$$$$00000004)
    .ARM.Collect$$$$00000007                 0x000000c8   Section        8  entry7.o(.ARM.Collect$$$$00000007)
    .ARM.Collect$$$$00002712                 0x000000d0   Section        4  entry2.o(.ARM.Collect$$$$00002712)
    __lit__00000000                          0x000000d0   Data           4  entry2.o(.ARM.Collect$$$$00002712)
    .text                                    0x000000d4   Section       28  startup_lpc11xx.o(.text)
    .text                                    0x000000f0   Section        0  system_lpc11xx.o(.text)
    .text                                    0x000001cc   Section        0  retarget.o(.text)
    .text                                    0x00000254   Section        0  tools.o(.text)
    .text                                    0x000002e8   Section        0  iusefp.o(.text)
    i.__0printf$bare                         0x000002e8   Section        0  printfb.o(i.__0printf$bare)
    .ARM.__at_0x02FC                         0x000002fc   Section        4  startup_lpc11xx.o(.ARM.__at_0x02FC)
    .text                                    0x00000300   Section        0  gpio.o(.text)
    NVIC_EnableIRQ                           0x000007c7   Thumb Code    14  gpio.o(.text)
    .text                                    0x000007e8   Section        0  uart.o(.text)
    .text                                    0x00000a34   Section        0  i2c.o(.text)
    .text                                    0x00000d3c   Section        0  adc.o(.text)
    .text                                    0x00000f00   Section        0  ssp.o(.text)
    NVIC_EnableIRQ                           0x000011f7   Thumb Code    14  ssp.o(.text)
    .text                                    0x00001230   Section        0  key.o(.text)
    .text                                    0x000012d8   Section        0  seg7led.o(.text)
    .text                                    0x00001368   Section        0  temp_hum.o(.text)
    .text                                    0x0000157c   Section        0  light.o(.text)
    readCommandReg                           0x0000157d   Thumb Code    32  light.o(.text)
    readControlReg                           0x0000159d   Thumb Code    32  light.o(.text)
    .text                                    0x0000186c   Section        0  acc.o(.text)
    getStatus                                0x0000186d   Thumb Code    32  acc.o(.text)
    getModeControl                           0x0000188d   Thumb Code    32  acc.o(.text)
    setModeControl                           0x000018ad   Thumb Code    24  acc.o(.text)
    .text                                    0x000019f0   Section        0  rfid.o(.text)
    .text                                    0x00001bd4   Section        0  spi_uart.o(.text)
    .text                                    0x00001ea4   Section      196  os_cpu_a.o(.text)
    .text                                    0x00001f68   Section        0  os_cpu_c.o(.text)
    .text                                    0x00002094   Section        0  os_core.o(.text)
    OS_SchedNew                              0x000021a1   Thumb Code    90  os_core.o(.text)
    OS_InitTaskStat                          0x00002661   Thumb Code    50  os_core.o(.text)
    OS_InitTaskIdle                          0x000026b5   Thumb Code    50  os_core.o(.text)
    OS_InitEventList                         0x000026f9   Thumb Code    78  os_core.o(.text)
    OS_InitTCBList                           0x00002747   Thumb Code    88  os_core.o(.text)
    OS_InitRdyList                           0x0000279f   Thumb Code    46  os_core.o(.text)
    OS_InitMisc                              0x000027cd   Thumb Code    44  os_core.o(.text)
    .text                                    0x00002e4c   Section        0  os_flag.o(.text)
    OS_FlagTaskRdy                           0x00002fc7   Thumb Code    92  os_flag.o(.text)
    OS_FlagBlock                             0x0000318b   Thumb Code   136  os_flag.o(.text)
    .text                                    0x00003640   Section        0  os_mbox.o(.text)
    .text                                    0x00003a38   Section        0  os_mem.o(.text)
    .text                                    0x00003bec   Section        0  os_q.o(.text)
    .text                                    0x000041c0   Section        0  os_sem.o(.text)
    .text                                    0x00004578   Section        0  os_task.o(.text)
    .text                                    0x00004ddc   Section        0  os_time.o(.text)
    .text                                    0x00004f98   Section        0  main.o(.text)
    NVIC_SetPriority                         0x00004f99   Thumb Code   110  main.o(.text)
    .text                                    0x0000550c   Section        0  lpc11c14_it.o(.text)
    .text                                    0x00005534   Section        0  crc16.o(.text)
    .text                                    0x00005570   Section        0  led_spk_fan_adc.o(.text)
    .text                                    0x000056c2   Section        0  uidiv.o(.text)
    .text                                    0x000056ee   Section        0  uldiv.o(.text)
    .text                                    0x00005750   Section        0  dadd.o(.text)
    .text                                    0x000058b4   Section        0  dmul.o(.text)
    .text                                    0x00005980   Section        0  ddiv.o(.text)
    .text                                    0x00005a70   Section        0  dfixul.o(.text)
    .text                                    0x00005ab0   Section       40  cdrcmple.o(.text)
    .text                                    0x00005ad8   Section       36  init.o(.text)
    .text                                    0x00005afc   Section        0  llshl.o(.text)
    .text                                    0x00005b1c   Section        0  llushr.o(.text)
    .text                                    0x00005b3e   Section        0  llsshr.o(.text)
    .text                                    0x00005b64   Section        0  depilogue.o(.text)
    i.__0vsnprintf                           0x00005c28   Section        0  printfa.o(i.__0vsnprintf)
    i.__ARM_clz                              0x00005c4c   Section        0  depilogue.o(i.__ARM_clz)
    i.__ARM_common_switch8                   0x00005c7a   Section        0  i2c.o(i.__ARM_common_switch8)
    i.__scatterload_copy                     0x00005c96   Section       14  handlers.o(i.__scatterload_copy)
    i.__scatterload_null                     0x00005ca4   Section        2  handlers.o(i.__scatterload_null)
    i.__scatterload_zeroinit                 0x00005ca6   Section       14  handlers.o(i.__scatterload_zeroinit)
    i._fp_digits                             0x00005cb4   Section        0  printfa.o(i._fp_digits)
    _fp_digits                               0x00005cb5   Thumb Code   312  printfa.o(i._fp_digits)
    i._printf_core                           0x00005e08   Section        0  printfb.o(i._printf_core)
    _printf_core                             0x00005e09   Thumb Code    30  printfb.o(i._printf_core)
    i._printf_core                           0x00005e28   Section        0  printfa.o(i._printf_core)
    _printf_core                             0x00005e29   Thumb Code  1774  printfa.o(i._printf_core)
    i._printf_post_padding                   0x00006528   Section        0  printfa.o(i._printf_post_padding)
    _printf_post_padding                     0x00006529   Thumb Code    32  printfa.o(i._printf_post_padding)
    i._printf_pre_padding                    0x00006548   Section        0  printfa.o(i._printf_pre_padding)
    _printf_pre_padding                      0x00006549   Thumb Code    42  printfa.o(i._printf_pre_padding)
    i._snputc                                0x00006572   Section        0  printfa.o(i._snputc)
    _snputc                                  0x00006573   Thumb Code    22  printfa.o(i._snputc)
    .constdata                               0x00006588   Section       16  gpio.o(.constdata)
    LPC_GPIO                                 0x00006588   Data          16  gpio.o(.constdata)
    .constdata                               0x00006598   Section       48  seg7led.o(.constdata)
    LPC_GPIO                                 0x00006598   Data          16  seg7led.o(.constdata)
    .constdata                               0x000065c8   Section       56  rfid.o(.constdata)
    LPC_GPIO                                 0x000065c8   Data          16  rfid.o(.constdata)
    .constdata                               0x00006600   Section      256  os_core.o(.constdata)
    .constdata                               0x00006700   Section      512  crc16.o(.constdata)
    crc16_table                              0x00006700   Data         512  crc16.o(.constdata)
    .data                                    0x10000000   Section       12  system_lpc11xx.o(.data)
    .data                                    0x1000000c   Section       44  gpio.o(.data)
    .data                                    0x10000038   Section       16  uart.o(.data)
    .data                                    0x10000048   Section        8  retarget.o(.data)
    .data                                    0x10000050   Section       41  i2c.o(.data)
    I2CMasterState                           0x10000050   Data           4  i2c.o(.data)
    I2CSlaveState                            0x10000054   Data           4  i2c.o(.data)
    I2CCount                                 0x10000058   Data           4  i2c.o(.data)
    RdIndex                                  0x1000005c   Data           4  i2c.o(.data)
    WrIndex                                  0x10000060   Data           4  i2c.o(.data)
    I2CMode                                  0x10000064   Data           4  i2c.o(.data)
    I2CMasterBuffer                          0x10000068   Data           4  i2c.o(.data)
    I2CSlaveBuffer                           0x1000006c   Data           4  i2c.o(.data)
    I2CReadLength                            0x10000070   Data           4  i2c.o(.data)
    I2CWriteLength                           0x10000074   Data           4  i2c.o(.data)
    I2CAddr                                  0x10000078   Data           1  i2c.o(.data)
    .data                                    0x1000007c   Section       24  ssp.o(.data)
    .data                                    0x10000094   Section        8  light.o(.data)
    range                                    0x10000094   Data           4  light.o(.data)
    width                                    0x10000098   Data           4  light.o(.data)
    .data                                    0x1000009c   Section        8  spi_uart.o(.data)
    .data                                    0x100000a4   Section       72  os_core.o(.data)
    .data                                    0x100000ec   Section       12  main.o(.data)
    .bss                                     0x100000f8   Section       64  uart.o(.bss)
    .bss                                     0x10000138   Section       32  adc.o(.bss)
    .bss                                     0x10000158   Section      256  spi_uart.o(.bss)
    .bss                                     0x10000258   Section     4188  os_core.o(.bss)
    .bss                                     0x100012b4   Section     2850  main.o(.bss)
    STACK                                    0x10001dd8   Section      256  startup_lpc11xx.o(STACK)

    Global Symbols

    Symbol Name                              Value     Ov Type        Size  Object(Section)

    BuildAttributes$$THM_ISAv3M$S$PE$A:L22$X:L11$S22$IEEE1$IW$USESV6$~STKCKD$USESV7$~SHL$OSPACE$ROPI$EBA8$MICROLIB$REQ8$PRES8$EABIv2 0x00000000   Number         0  anon$$obj.o ABSOLUTE
    __ARM_use_no_argv                        0x00000000   Number         0  main.o ABSOLUTE
    __Vectors                                0x00000000   Data           4  startup_lpc11xx.o(RESET)
    __use_no_errno                           0x00000000   Number         0  useno.o ABSOLUTE
    __use_no_exception_handling              0x00000000   Number         0  useno.o ABSOLUTE
    __use_no_fp                              0x00000000   Number         0  useno.o ABSOLUTE
    __use_no_heap                            0x00000000   Number         0  useno.o ABSOLUTE
    __use_no_heap_region                     0x00000000   Number         0  useno.o ABSOLUTE
    __use_no_semihosting                     0x00000000   Number         0  useno.o ABSOLUTE
    __use_no_semihosting_swi                 0x00000000   Number         0  useno.o ABSOLUTE
    __use_no_signal_handling                 0x00000000   Number         0  useno.o ABSOLUTE
    __decompress                              - Undefined Weak Reference
    __main                                   0x000000c1   Thumb Code     0  entry.o(.ARM.Collect$$$$00000000)
    _main_stk                                0x000000c1   Thumb Code     0  entry2.o(.ARM.Collect$$$$00000001)
    _main_scatterload                        0x000000c5   Thumb Code     0  entry5.o(.ARM.Collect$$$$00000004)
    __main_after_scatterload                 0x000000c9   Thumb Code     0  entry5.o(.ARM.Collect$$$$00000004)
    _main_init                               0x000000c9   Thumb Code     0  entry7.o(.ARM.Collect$$$$00000007)
    Reset_Handler                            0x000000d5   Thumb Code     4  startup_lpc11xx.o(.text)
    ADC_IRQHandler                           0x000000eb   Thumb Code     0  startup_lpc11xx.o(.text)
    BOD_IRQHandler                           0x000000eb   Thumb Code     0  startup_lpc11xx.o(.text)
    CAN_IRQHandler                           0x000000eb   Thumb Code     0  startup_lpc11xx.o(.text)
    FMC_IRQHandler                           0x000000eb   Thumb Code     0  startup_lpc11xx.o(.text)
    TIMER16_0_IRQHandler                     0x000000eb   Thumb Code     0  startup_lpc11xx.o(.text)
    TIMER16_1_IRQHandler                     0x000000eb   Thumb Code     0  startup_lpc11xx.o(.text)
    TIMER32_0_IRQHandler                     0x000000eb   Thumb Code     0  startup_lpc11xx.o(.text)
    TIMER32_1_IRQHandler                     0x000000eb   Thumb Code     0  startup_lpc11xx.o(.text)
    USB_FIQHandler                           0x000000eb   Thumb Code     0  startup_lpc11xx.o(.text)
    USB_IRQHandler                           0x000000eb   Thumb Code     0  startup_lpc11xx.o(.text)
    WAKEUP_IRQHandler                        0x000000eb   Thumb Code     0  startup_lpc11xx.o(.text)
    WDT_IRQHandler                           0x000000eb   Thumb Code     0  startup_lpc11xx.o(.text)
    Main_PLL_Setup                           0x000000f1   Thumb Code   136  system_lpc11xx.o(.text)
    SystemInit                               0x00000179   Thumb Code    60  system_lpc11xx.o(.text)
    PutCh                                    0x000001cd   Thumb Code    18  retarget.o(.text)
    fputc                                    0x000001df   Thumb Code    14  retarget.o(.text)
    GetCh                                    0x000001ed   Thumb Code    34  retarget.o(.text)
    fgetc                                    0x0000020f   Thumb Code    16  retarget.o(.text)
    _ttywrch                                 0x0000021f   Thumb Code    12  retarget.o(.text)
    ferror                                   0x0000022b   Thumb Code     8  retarget.o(.text)
    _sys_exit                                0x00000233   Thumb Code     4  retarget.o(.text)
    GetCh_NoIRQ                              0x00000237   Thumb Code    18  retarget.o(.text)
    delay_ms                                 0x00000255   Thumb Code   140  tools.o(.text)
    __0printf$bare                           0x000002e9   Thumb Code    12  printfb.o(i.__0printf$bare)
    __1printf$bare                           0x000002e9   Thumb Code     0  printfb.o(i.__0printf$bare)
    __2printf                                0x000002e9   Thumb Code     0  printfb.o(i.__0printf$bare)
    __I$use$fp                               0x000002e9   Thumb Code     0  iusefp.o(.text)
    GPIOIntClear                             0x00000301   Thumb Code    88  gpio.o(.text)
    GPIOIntStatus                            0x00000359   Thumb Code    94  gpio.o(.text)
    PIOINT0_IRQHandler                       0x000003b7   Thumb Code    46  gpio.o(.text)
    PIOINT1_IRQHandler                       0x000003e5   Thumb Code    46  gpio.o(.text)
    GPIOSetValue                             0x00000413   Thumb Code    22  gpio.o(.text)
    PIOINT2_IRQHandler                       0x00000429   Thumb Code    46  gpio.o(.text)
    PIOINT3_IRQHandler                       0x00000457   Thumb Code    66  gpio.o(.text)
    GPIOInit                                 0x00000499   Thumb Code    40  gpio.o(.text)
    GPIOSetInterrupt                         0x000004c1   Thumb Code   446  gpio.o(.text)
    GPIOIntEnable                            0x0000067f   Thumb Code    88  gpio.o(.text)
    GPIOIntDisable                           0x000006d7   Thumb Code   144  gpio.o(.text)
    GPIOGetValue                             0x00000767   Thumb Code    18  gpio.o(.text)
    GPIOSetDir                               0x00000779   Thumb Code    78  gpio.o(.text)
    UART_IRQHandler                          0x000007e9   Thumb Code   180  uart.o(.text)
    UARTInit                                 0x0000089d   Thumb Code   202  uart.o(.text)
    UARTSend                                 0x00000967   Thumb Code    30  uart.o(.text)
    UART0_PutChar                            0x00000985   Thumb Code    18  uart.o(.text)
    UART0_PutString                          0x00000997   Thumb Code    22  uart.o(.text)
    UART0_printf                             0x000009ad   Thumb Code    40  uart.o(.text)
    UART0_GetChar                            0x000009d5   Thumb Code    54  uart.o(.text)
    I2C_IRQHandler                           0x00000a35   Thumb Code   394  i2c.o(.text)
    I2CStart                                 0x00000bbf   Thumb Code    42  i2c.o(.text)
    I2CStop                                  0x00000be9   Thumb Code    28  i2c.o(.text)
    I2CInit                                  0x00000c05   Thumb Code   122  i2c.o(.text)
    I2CEngine                                0x00000c7f   Thumb Code    56  i2c.o(.text)
    I2CRead                                  0x00000cb7   Thumb Code    46  i2c.o(.text)
    I2CWrite                                 0x00000ce5   Thumb Code    40  i2c.o(.text)
    ADCInit_NXP                              0x00000d3d   Thumb Code   150  adc.o(.text)
    ADCInit                                  0x00000dd3   Thumb Code   126  adc.o(.text)
    ADCRead                                  0x00000e51   Thumb Code    98  adc.o(.text)
    ADCBurstRead                             0x00000eb3   Thumb Code    50  adc.o(.text)
    SSP0_IRQHandler                          0x00000f01   Thumb Code    66  ssp.o(.text)
    SSP1_IRQHandler                          0x00000f43   Thumb Code    66  ssp.o(.text)
    SPI_IOConfig                             0x00000f85   Thumb Code   392  ssp.o(.text)
    SPI_Init                                 0x0000110d   Thumb Code   124  ssp.o(.text)
    SPI_PutGet                               0x00001189   Thumb Code   110  ssp.o(.text)
    KEY_Init                                 0x00001231   Thumb Code    64  key.o(.text)
    KEY_Read                                 0x00001271   Thumb Code   102  key.o(.text)
    Seg7Led_Init                             0x000012d9   Thumb Code    54  seg7led.o(.text)
    Seg7Led_Put                              0x0000130f   Thumb Code    86  seg7led.o(.text)
    Read_Temp_Hum                            0x00001369   Thumb Code   458  temp_hum.o(.text)
    Temp_Hum_Collect                         0x00001533   Thumb Code    58  temp_hum.o(.text)
    light_init                               0x000015bd   Thumb Code     2  light.o(.text)
    light_enable                             0x000015bf   Thumb Code    38  light.o(.text)
    light_read                               0x000015e5   Thumb Code    86  light.o(.text)
    light_setMode                            0x0000163b   Thumb Code    44  light.o(.text)
    light_setWidth                           0x00001667   Thumb Code    98  light.o(.text)
    light_setRange                           0x000016c9   Thumb Code    96  light.o(.text)
    light_setHiThreshold                     0x00001729   Thumb Code    50  light.o(.text)
    light_setLoThreshold                     0x0000175b   Thumb Code    50  light.o(.text)
    light_setIrqInCycles                     0x0000178d   Thumb Code    44  light.o(.text)
    light_getIrqStatus                       0x000017b9   Thumb Code    16  light.o(.text)
    light_clearIrqStatus                     0x000017c9   Thumb Code    36  light.o(.text)
    light_shutdown                           0x000017ed   Thumb Code    62  light.o(.text)
    Light_Collect                            0x0000182b   Thumb Code    40  light.o(.text)
    acc_init                                 0x000018c5   Thumb Code    10  acc.o(.text)
    acc_read                                 0x000018cf   Thumb Code   118  acc.o(.text)
    acc_setRange                             0x00001945   Thumb Code    34  acc.o(.text)
    acc_setMode                              0x00001967   Thumb Code    30  acc.o(.text)
    Axis3_Collect                            0x00001985   Thumb Code   106  acc.o(.text)
    RFID_CheckSum                            0x000019f1   Thumb Code    50  rfid.o(.text)
    RFID_Operate                             0x00001a23   Thumb Code   314  rfid.o(.text)
    RFID_Collect                             0x00001b5d   Thumb Code   116  rfid.o(.text)
    SPI752_RegRead                           0x00001bd5   Thumb Code    58  spi_uart.o(.text)
    ZigBee_IRQ_Process                       0x00001c0f   Thumb Code   150  spi_uart.o(.text)
    SPI752_RegWrite                          0x00001ca5   Thumb Code    52  spi_uart.o(.text)
    SPI752_Init                              0x00001cd9   Thumb Code   216  spi_uart.o(.text)
    SPI752_PutChar                           0x00001db1   Thumb Code    34  spi_uart.o(.text)
    ZigBee_PutChar                           0x00001dd3   Thumb Code    14  spi_uart.o(.text)
    ZigBee_Send                              0x00001de1   Thumb Code    26  spi_uart.o(.text)
    ZigBee_PutString                         0x00001dfb   Thumb Code    24  spi_uart.o(.text)
    SPI752_GetChar                           0x00001e13   Thumb Code   106  spi_uart.o(.text)
    ZigBee_GetChar                           0x00001e7d   Thumb Code    14  spi_uart.o(.text)
    OS_CPU_SR_Save                           0x00001ea5   Thumb Code     0  os_cpu_a.o(.text)
    OS_CPU_SR_Restore                        0x00001ead   Thumb Code     0  os_cpu_a.o(.text)
    OSStartHighRdy                           0x00001eb3   Thumb Code     0  os_cpu_a.o(.text)
    OSCtxSw                                  0x00001ed3   Thumb Code     0  os_cpu_a.o(.text)
    OSIntCtxSw                               0x00001edb   Thumb Code     0  os_cpu_a.o(.text)
    OS_CPU_PendSVHandler                     0x00001ee3   Thumb Code     0  os_cpu_a.o(.text)
    OSInitHookBegin                          0x00001f69   Thumb Code     2  os_cpu_c.o(.text)
    OSInitHookEnd                            0x00001f6b   Thumb Code     2  os_cpu_c.o(.text)
    OSTaskCreateHook                         0x00001f6d   Thumb Code     2  os_cpu_c.o(.text)
    OSTaskDelHook                            0x00001f6f   Thumb Code     2  os_cpu_c.o(.text)
    OSTaskIdleHook                           0x00001f71   Thumb Code     2  os_cpu_c.o(.text)
    OSTaskStatHook                           0x00001f73   Thumb Code     2  os_cpu_c.o(.text)
    OSTaskStkInit                            0x00001f75   Thumb Code   132  os_cpu_c.o(.text)
    OSTaskSwHook                             0x00001ff9   Thumb Code     2  os_cpu_c.o(.text)
    OSTCBInitHook                            0x00001ffb   Thumb Code     2  os_cpu_c.o(.text)
    OSTimeTickHook                           0x00001ffd   Thumb Code     2  os_cpu_c.o(.text)
    OS_CPU_SysTickHandler                    0x00001fff   Thumb Code    34  os_cpu_c.o(.text)
    OS_CPU_SysTickInit                       0x00002021   Thumb Code    54  os_cpu_c.o(.text)
    OS_StrLen                                0x00002095   Thumb Code    20  os_core.o(.text)
    OSEventNameGet                           0x000020a9   Thumb Code    96  os_core.o(.text)
    OSEventNameSet                           0x00002109   Thumb Code    82  os_core.o(.text)
    OS_EventTaskRemoveMulti                  0x0000215b   Thumb Code    70  os_core.o(.text)
    OS_Sched                                 0x000021fb   Thumb Code    92  os_core.o(.text)
    OS_EventTaskWaitMulti                    0x00002257   Thumb Code   140  os_core.o(.text)
    OSEventPendMulti                         0x000022e3   Thumb Code   720  os_core.o(.text)
    OS_TaskStatStkChk                        0x000025b3   Thumb Code    58  os_core.o(.text)
    OS_TaskStat                              0x000025ed   Thumb Code   116  os_core.o(.text)
    OS_TaskIdle                              0x00002693   Thumb Code    34  os_core.o(.text)
    OS_MemClr                                0x000026e7   Thumb Code    18  os_core.o(.text)
    OSInit                                   0x000027f9   Thumb Code    48  os_core.o(.text)
    OSIntEnter                               0x00002829   Thumb Code    28  os_core.o(.text)
    OSIntExit                                0x00002845   Thumb Code   268  os_core.o(.text)
    OSSchedLock                              0x00002951   Thumb Code    52  os_core.o(.text)
    OSSchedUnlock                            0x00002985   Thumb Code    88  os_core.o(.text)
    OSStart                                  0x000029dd   Thumb Code    50  os_core.o(.text)
    OSStatInit                               0x00002a0f   Thumb Code    62  os_core.o(.text)
    OSTimeTick                               0x00002a4d   Thumb Code   224  os_core.o(.text)
    OSVersion                                0x00002b2d   Thumb Code     6  os_core.o(.text)
    OS_Dummy                                 0x00002b33   Thumb Code     2  os_core.o(.text)
    OS_EventTaskRemove                       0x00002b35   Thumb Code    48  os_core.o(.text)
    OS_EventTaskRdy                          0x00002b65   Thumb Code   190  os_core.o(.text)
    OS_EventTaskWait                         0x00002c23   Thumb Code   116  os_core.o(.text)
    OS_EventWaitListInit                     0x00002c97   Thumb Code    32  os_core.o(.text)
    OS_MemCopy                               0x00002cb7   Thumb Code    20  os_core.o(.text)
    OS_TCBInit                               0x00002ccb   Thumb Code   360  os_core.o(.text)
    OSFlagAccept                             0x00002e4d   Thumb Code   250  os_flag.o(.text)
    OSFlagCreate                             0x00002f47   Thumb Code    86  os_flag.o(.text)
    OS_FlagUnlink                            0x00002f9d   Thumb Code    42  os_flag.o(.text)
    OSFlagDel                                0x00003023   Thumb Code   218  os_flag.o(.text)
    OSFlagNameGet                            0x000030fd   Thumb Code    78  os_flag.o(.text)
    OSFlagNameSet                            0x0000314b   Thumb Code    64  os_flag.o(.text)
    OSFlagPend                               0x00003213   Thumb Code   608  os_flag.o(.text)
    OSFlagPendGetFlagsRdy                    0x00003473   Thumb Code    26  os_flag.o(.text)
    OSFlagPost                               0x0000348d   Thumb Code   304  os_flag.o(.text)
    OSFlagQuery                              0x000035bd   Thumb Code    44  os_flag.o(.text)
    OS_FlagInit                              0x000035e9   Thumb Code    70  os_flag.o(.text)
    OSMboxAccept                             0x00003641   Thumb Code    38  os_mbox.o(.text)
    OSMboxCreate                             0x00003667   Thumb Code    78  os_mbox.o(.text)
    OSMboxDel                                0x000036b5   Thumb Code   212  os_mbox.o(.text)
    OSMboxPend                               0x00003789   Thumb Code   258  os_mbox.o(.text)
    OSMboxPendAbort                          0x0000388b   Thumb Code   128  os_mbox.o(.text)
    OSMboxPost                               0x0000390b   Thumb Code    84  os_mbox.o(.text)
    OSMboxPostOpt                            0x0000395f   Thumb Code   120  os_mbox.o(.text)
    OSMboxQuery                              0x000039d7   Thumb Code    78  os_mbox.o(.text)
    OSMemCreate                              0x00003a39   Thumb Code   124  os_mem.o(.text)
    OSMemGet                                 0x00003ab5   Thumb Code    60  os_mem.o(.text)
    OSMemNameGet                             0x00003af1   Thumb Code    58  os_mem.o(.text)
    OSMemNameSet                             0x00003b2b   Thumb Code    46  os_mem.o(.text)
    OSMemPut                                 0x00003b59   Thumb Code    54  os_mem.o(.text)
    OSMemQuery                               0x00003b8f   Thumb Code    52  os_mem.o(.text)
    OS_MemInit                               0x00003bc3   Thumb Code    24  os_mem.o(.text)
    OSQAccept                                0x00003bed   Thumb Code    86  os_q.o(.text)
    OSQCreate                                0x00003c43   Thumb Code   148  os_q.o(.text)
    OSQDel                                   0x00003cd7   Thumb Code   244  os_q.o(.text)
    OSQFlush                                 0x00003dcb   Thumb Code    36  os_q.o(.text)
    OSQPend                                  0x00003def   Thumb Code   286  os_q.o(.text)
    OSQPendAbort                             0x00003f0d   Thumb Code   128  os_q.o(.text)
    OSQPost                                  0x00003f8d   Thumb Code   112  os_q.o(.text)
    OSQPostFront                             0x00003ffd   Thumb Code   138  os_q.o(.text)
    OSQPostOpt                               0x00004087   Thumb Code   180  os_q.o(.text)
    OSQQuery                                 0x0000413b   Thumb Code   112  os_q.o(.text)
    OS_QInit                                 0x000041ab   Thumb Code    14  os_q.o(.text)
    OSSemAccept                              0x000041c1   Thumb Code    44  os_sem.o(.text)
    OSSemCreate                              0x000041ed   Thumb Code    78  os_sem.o(.text)
    OSSemDel                                 0x0000423b   Thumb Code   212  os_sem.o(.text)
    OSSemPend                                0x0000430f   Thumb Code   234  os_sem.o(.text)
    OSSemPendAbort                           0x000043f9   Thumb Code   128  os_sem.o(.text)
    OSSemPost                                0x00004479   Thumb Code    88  os_sem.o(.text)
    OSSemQuery                               0x000044d1   Thumb Code    78  os_sem.o(.text)
    OSSemSet                                 0x0000451f   Thumb Code    66  os_sem.o(.text)
    OSTaskChangePrio                         0x00004579   Thumb Code   446  os_task.o(.text)
    OSTaskCreate                             0x00004737   Thumb Code   150  os_task.o(.text)
    OS_TaskStkClr                            0x000047cd   Thumb Code    26  os_task.o(.text)
    OSTaskCreateExt                          0x000047e7   Thumb Code   160  os_task.o(.text)
    OSTaskDel                                0x00004887   Thumb Code   358  os_task.o(.text)
    OSTaskDelReq                             0x000049ed   Thumb Code    98  os_task.o(.text)
    OSTaskNameGet                            0x00004a4f   Thumb Code   114  os_task.o(.text)
    OSTaskNameSet                            0x00004ac1   Thumb Code    98  os_task.o(.text)
    OSTaskResume                             0x00004b23   Thumb Code   166  os_task.o(.text)
    OSTaskStkChk                             0x00004bc9   Thumb Code   130  os_task.o(.text)
    OSTaskSuspend                            0x00004c4b   Thumb Code   154  os_task.o(.text)
    OSTaskQuery                              0x00004ce5   Thumb Code    80  os_task.o(.text)
    OSTaskRegGet                             0x00004d35   Thumb Code    58  os_task.o(.text)
    OSTaskRegSet                             0x00004d6f   Thumb Code    98  os_task.o(.text)
    OS_TaskReturn                            0x00004dd1   Thumb Code    10  os_task.o(.text)
    OSTimeDly                                0x00004ddd   Thumb Code   110  os_time.o(.text)
    OSTimeDlyHMSM                            0x00004e4b   Thumb Code    82  os_time.o(.text)
    OSTimeDlyResume                          0x00004e9d   Thumb Code   176  os_time.o(.text)
    OSTimeGet                                0x00004f4d   Thumb Code    24  os_time.o(.text)
    OSTimeSet                                0x00004f65   Thumb Code    24  os_time.o(.text)
    Task_Send                                0x00005007   Thumb Code    40  main.o(.text)
    Task_RFid                                0x0000502f   Thumb Code   116  main.o(.text)
    Task_ACC                                 0x000050a3   Thumb Code    28  main.o(.text)
    Task_ADC                                 0x000050bf   Thumb Code    30  main.o(.text)
    Task_Light                               0x000050dd   Thumb Code    38  main.o(.text)
    Task_Temp_Hum                            0x00005103   Thumb Code    24  main.o(.text)
    Task_BeepFan                             0x0000511b   Thumb Code    76  main.o(.text)
    Task_Key                                 0x00005167   Thumb Code    42  main.o(.text)
    Task_Seg7Led                             0x00005191   Thumb Code    36  main.o(.text)
    Task_Led                                 0x000051b5   Thumb Code    96  main.o(.text)
    Task_Start                               0x00005215   Thumb Code    20  main.o(.text)
    main                                     0x00005229   Thumb Code   678  main.o(.text)
    NMI_Handler                              0x0000550d   Thumb Code     2  lpc11c14_it.o(.text)
    HardFault_Handler                        0x0000550f   Thumb Code     4  lpc11c14_it.o(.text)
    MemManage_Handler                        0x00005513   Thumb Code     4  lpc11c14_it.o(.text)
    BusFault_Handler                         0x00005517   Thumb Code     4  lpc11c14_it.o(.text)
    UsageFault_Handler                       0x0000551b   Thumb Code     4  lpc11c14_it.o(.text)
    SVC_Handler                              0x0000551f   Thumb Code     2  lpc11c14_it.o(.text)
    DebugMon_Handler                         0x00005521   Thumb Code     2  lpc11c14_it.o(.text)
    PendSV_Handler                           0x00005523   Thumb Code     8  lpc11c14_it.o(.text)
    SysTick_Handler                          0x0000552b   Thumb Code     8  lpc11c14_it.o(.text)
    crc16                                    0x00005535   Thumb Code    22  crc16.o(.text)
    make_crc16                               0x0000554b   Thumb Code    34  crc16.o(.text)
    ADC_Collect                              0x00005571   Thumb Code    26  led_spk_fan_adc.o(.text)
    send_package                             0x0000558b   Thumb Code   312  led_spk_fan_adc.o(.text)
    __aeabi_uidiv                            0x000056c3   Thumb Code     0  uidiv.o(.text)
    __aeabi_uidivmod                         0x000056c3   Thumb Code    44  uidiv.o(.text)
    __aeabi_uldivmod                         0x000056ef   Thumb Code    96  uldiv.o(.text)
    __aeabi_dadd                             0x00005751   Thumb Code   326  dadd.o(.text)
    __aeabi_dsub                             0x00005897   Thumb Code    12  dadd.o(.text)
    __aeabi_drsub                            0x000058a3   Thumb Code    12  dadd.o(.text)
    __aeabi_dmul                             0x000058b5   Thumb Code   198  dmul.o(.text)
    __aeabi_ddiv                             0x00005981   Thumb Code   234  ddiv.o(.text)
    __aeabi_d2ulz                            0x00005a71   Thumb Code    54  dfixul.o(.text)
    __aeabi_cdrcmple                         0x00005ab1   Thumb Code    38  cdrcmple.o(.text)
    __scatterload                            0x00005ad9   Thumb Code    28  init.o(.text)
    __scatterload_rt2                        0x00005ad9   Thumb Code     0  init.o(.text)
    __aeabi_llsl                             0x00005afd   Thumb Code    32  llshl.o(.text)
    _ll_shift_l                              0x00005afd   Thumb Code     0  llshl.o(.text)
    __aeabi_llsr                             0x00005b1d   Thumb Code    34  llushr.o(.text)
    _ll_ushift_r                             0x00005b1d   Thumb Code     0  llushr.o(.text)
    __aeabi_lasr                             0x00005b3f   Thumb Code    38  llsshr.o(.text)
    _ll_sshift_r                             0x00005b3f   Thumb Code     0  llsshr.o(.text)
    _double_round                            0x00005b65   Thumb Code    26  depilogue.o(.text)
    _double_epilogue                         0x00005b7f   Thumb Code   170  depilogue.o(.text)
    __0vsnprintf                             0x00005c29   Thumb Code    32  printfa.o(i.__0vsnprintf)
    __1vsnprintf                             0x00005c29   Thumb Code     0  printfa.o(i.__0vsnprintf)
    __2vsnprintf                             0x00005c29   Thumb Code     0  printfa.o(i.__0vsnprintf)
    __c89vsnprintf                           0x00005c29   Thumb Code     0  printfa.o(i.__0vsnprintf)
    vsnprintf                                0x00005c29   Thumb Code     0  printfa.o(i.__0vsnprintf)
    __ARM_clz                                0x00005c4d   Thumb Code    46  depilogue.o(i.__ARM_clz)
    __ARM_common_switch8                     0x00005c7b   Thumb Code    28  i2c.o(i.__ARM_common_switch8)
    __scatterload_copy                       0x00005c97   Thumb Code    14  handlers.o(i.__scatterload_copy)
    __scatterload_null                       0x00005ca5   Thumb Code     2  handlers.o(i.__scatterload_null)
    __scatterload_zeroinit                   0x00005ca7   Thumb Code    14  handlers.o(i.__scatterload_zeroinit)
    segcode                                  0x000065a8   Data          32  seg7led.o(.constdata)
    RFID_READ_MOD_TYPE_01                    0x000065d8   Data           2  rfid.o(.constdata)
    RFID_READ_CARD_20                        0x000065da   Data           2  rfid.o(.constdata)
    RFID_READ_DATA_BLOCK_21                  0x000065dc   Data          10  rfid.o(.constdata)
    RFID_WRITE_DATA_BLOCK_22                 0x000065e6   Data          26  rfid.o(.constdata)
    OSUnMapTbl                               0x00006600   Data         256  os_core.o(.constdata)
    Region$$Table$$Base                      0x00006900   Number         0  anon$$obj.o(Region$$Table)
    Region$$Table$$Limit                     0x00006920   Number         0  anon$$obj.o(Region$$Table)
    ClockSource                              0x10000000   Data           4  system_lpc11xx.o(.data)
    SystemFrequency                          0x10000004   Data           4  system_lpc11xx.o(.data)
    SystemAHBFrequency                       0x10000008   Data           4  system_lpc11xx.o(.data)
    gpio0_counter                            0x1000000c   Data           4  gpio.o(.data)
    p0_1_counter                             0x10000010   Data           4  gpio.o(.data)
    gpio1_counter                            0x10000014   Data           4  gpio.o(.data)
    p1_1_counter                             0x10000018   Data           4  gpio.o(.data)
    gpio2_counter                            0x1000001c   Data           4  gpio.o(.data)
    p2_1_counter                             0x10000020   Data           4  gpio.o(.data)
    gpio3_counter                            0x10000024   Data           4  gpio.o(.data)
    p3_1_counter                             0x10000028   Data           4  gpio.o(.data)
    p3_2_counter                             0x1000002c   Data           4  gpio.o(.data)
    p2_8_counter                             0x10000030   Data           4  gpio.o(.data)
    p3_2_tc                                  0x10000034   Data           4  gpio.o(.data)
    UARTTxEmpty                              0x10000038   Data           1  uart.o(.data)
    UARTCount                                0x1000003c   Data           4  uart.o(.data)
    UART_op                                  0x10000040   Data           4  uart.o(.data)
    UARTStatus                               0x10000044   Data           4  uart.o(.data)
    __stdout                                 0x10000048   Data           4  retarget.o(.data)
    __stdin                                  0x1000004c   Data           4  retarget.o(.data)
    interruptRxStat0                         0x1000007c   Data           4  ssp.o(.data)
    interruptOverRunStat0                    0x10000080   Data           4  ssp.o(.data)
    interruptRxTimeoutStat0                  0x10000084   Data           4  ssp.o(.data)
    interruptRxStat1                         0x10000088   Data           4  ssp.o(.data)
    interruptOverRunStat1                    0x1000008c   Data           4  ssp.o(.data)
    interruptRxTimeoutStat1                  0x10000090   Data           4  ssp.o(.data)
    SPI752_rbuf_0_ip                         0x1000009c   Data           2  spi_uart.o(.data)
    SPI752_rbuf_0_op                         0x1000009e   Data           2  spi_uart.o(.data)
    SPI752_rbuf_1_ip                         0x100000a0   Data           2  spi_uart.o(.data)
    SPI752_rbuf_1_op                         0x100000a2   Data           2  spi_uart.o(.data)
    OSCtxSwCtr                               0x100000a4   Data           4  os_core.o(.data)
    OSEventFreeList                          0x100000a8   Data           4  os_core.o(.data)
    OSFlagFreeList                           0x100000ac   Data           4  os_core.o(.data)
    OSCPUUsage                               0x100000b0   Data           1  os_core.o(.data)
    OSIdleCtrMax                             0x100000b4   Data           4  os_core.o(.data)
    OSIdleCtrRun                             0x100000b8   Data           4  os_core.o(.data)
    OSStatRdy                                0x100000bc   Data           1  os_core.o(.data)
    OSIntNesting                             0x100000bd   Data           1  os_core.o(.data)
    OSLockNesting                            0x100000be   Data           1  os_core.o(.data)
    OSPrioCur                                0x100000bf   Data           1  os_core.o(.data)
    OSPrioHighRdy                            0x100000c0   Data           1  os_core.o(.data)
    OSRdyGrp                                 0x100000c2   Data           2  os_core.o(.data)
    OSRunning                                0x100000c4   Data           1  os_core.o(.data)
    OSTaskCtr                                0x100000c5   Data           1  os_core.o(.data)
    OSIdleCtr                                0x100000c8   Data           4  os_core.o(.data)
    OSTCBCur                                 0x100000cc   Data           4  os_core.o(.data)
    OSTCBFreeList                            0x100000d0   Data           4  os_core.o(.data)
    OSTCBHighRdy                             0x100000d4   Data           4  os_core.o(.data)
    OSTCBList                                0x100000d8   Data           4  os_core.o(.data)
    OSTickStepState                          0x100000dc   Data           1  os_core.o(.data)
    OSMemFreeList                            0x100000e0   Data           4  os_core.o(.data)
    OSQFreeList                              0x100000e4   Data           4  os_core.o(.data)
    OSTime                                   0x100000e8   Data           4  os_core.o(.data)
    dev_info                                 0x100000ec   Data           4  main.o(.data)
    Key_Sem                                  0x100000f0   Data           4  main.o(.data)
    Led_Mbox                                 0x100000f4   Data           4  main.o(.data)
    UARTBuffer                               0x100000f8   Data          64  uart.o(.bss)
    ADCValue                                 0x10000138   Data          32  adc.o(.bss)
    SPI752_rbuf_0                            0x10000158   Data         128  spi_uart.o(.bss)
    SPI752_rbuf_1                            0x100001d8   Data         128  spi_uart.o(.bss)
    OSEventTbl                               0x10000258   Data         480  os_core.o(.bss)
    OSFlagTbl                                0x10000438   Data          80  os_core.o(.bss)
    OSTaskStatStk                            0x10000488   Data         256  os_core.o(.bss)
    OSRdyTbl                                 0x10000588   Data          32  os_core.o(.bss)
    OSTaskIdleStk                            0x100005a8   Data         256  os_core.o(.bss)
    OSTCBPrioTbl                             0x100006a8   Data        1012  os_core.o(.bss)
    OSTCBTbl                                 0x10000a9c   Data        2024  os_core.o(.bss)
    OSMemTbl                                 0x10001284   Data          24  os_core.o(.bss)
    OSQTbl                                   0x1000129c   Data          24  os_core.o(.bss)
    Task_Start_STK                           0x100012b4   Data         256  main.o(.bss)
    Task_Led_STK                             0x100013b4   Data         256  main.o(.bss)
    Task_Seg7Led_STK                         0x100014b4   Data         256  main.o(.bss)
    Task_Key_STK                             0x100015b4   Data         256  main.o(.bss)
    Task_BeepFan_STK                         0x100016b4   Data         256  main.o(.bss)
    Task_Temp_Hum_STK                        0x100017b4   Data         256  main.o(.bss)
    Task_Light_STK                           0x100018b4   Data         256  main.o(.bss)
    Task_ADC_STK                             0x100019b4   Data         256  main.o(.bss)
    Task_ACC_STK                             0x10001ab4   Data         256  main.o(.bss)
    Task_RFid_STK                            0x10001bb4   Data         256  main.o(.bss)
    Task_Send_STK                            0x10001cb4   Data         256  main.o(.bss)
    dev                                      0x10001db4   Data          34  main.o(.bss)
    __initial_sp                             0x10001ed8   Data           0  startup_lpc11xx.o(STACK)



==============================================================================

Memory Map of the image

  Image Entry point : 0x000000c1

  Load Region LR_IROM1 (Base: 0x00000000, Size: 0x00006a18, Max: 0x00008000, ABSOLUTE)

    Execution Region ER_IROM1 (Base: 0x00000000, Size: 0x00006920, Max: 0x00008000, ABSOLUTE)

    Base Addr    Size         Type   Attr      Idx    E Section Name        Object

    0x00000000   0x000000c0   Data   RO            3    RESET               startup_lpc11xx.o
    0x000000c0   0x00000000   Code   RO          598  * .ARM.Collect$$$$00000000  mc_p.l(entry.o)
    0x000000c0   0x00000004   Code   RO          863    .ARM.Collect$$$$00000001  mc_p.l(entry2.o)
    0x000000c4   0x00000004   Code   RO          866    .ARM.Collect$$$$00000004  mc_p.l(entry5.o)
    0x000000c8   0x00000008   Code   RO          867    .ARM.Collect$$$$00000007  mc_p.l(entry7.o)
    0x000000d0   0x00000004   Code   RO          864    .ARM.Collect$$$$00002712  mc_p.l(entry2.o)
    0x000000d4   0x0000001c   Code   RO            5    .text               startup_lpc11xx.o
    0x000000f0   0x000000dc   Code   RO           27    .text               system_lpc11xx.o
    0x000001cc   0x00000088   Code   RO          125    .text               retarget.o
    0x00000254   0x00000094   Code   RO          215    .text               tools.o
    0x000002e8   0x00000000   Code   RO          870    .text               mc_p.l(iusefp.o)
    0x000002e8   0x00000014   Code   RO          604    i.__0printf$bare    mc_p.l(printfb.o)
    0x000002fc   0x00000004   Code   RO            4    .ARM.__at_0x02FC    startup_lpc11xx.o
    0x00000300   0x000004e8   Code   RO           51    .text               gpio.o
    0x000007e8   0x0000024c   Code   RO           96    .text               uart.o
    0x00000a34   0x00000308   Code   RO          148    .text               i2c.o
    0x00000d3c   0x000001c4   Code   RO          176    .text               adc.o
    0x00000f00   0x00000330   Code   RO          195    .text               ssp.o
    0x00001230   0x000000a6   Code   RO          239    .text               key.o
    0x000012d6   0x00000002   PAD
    0x000012d8   0x00000090   Code   RO          256    .text               seg7led.o
    0x00001368   0x00000214   Code   RO          274    .text               temp_hum.o
    0x0000157c   0x000002f0   Code   RO          295    .text               light.o
    0x0000186c   0x00000182   Code   RO          313    .text               acc.o
    0x000019ee   0x00000002   PAD
    0x000019f0   0x000001e4   Code   RO          328    .text               rfid.o
    0x00001bd4   0x000002d0   Code   RO          349    .text               spi_uart.o
    0x00001ea4   0x000000c4   Code   RO          366    .text               os_cpu_a.o
    0x00001f68   0x0000012c   Code   RO          369    .text               os_cpu_c.o
    0x00002094   0x00000db8   Code   RO          394    .text               os_core.o
    0x00002e4c   0x000007f4   Code   RO          423    .text               os_flag.o
    0x00003640   0x000003f8   Code   RO          435    .text               os_mbox.o
    0x00003a38   0x000001b4   Code   RO          447    .text               os_mem.o
    0x00003bec   0x000005d4   Code   RO          471    .text               os_q.o
    0x000041c0   0x000003b8   Code   RO          483    .text               os_sem.o
    0x00004578   0x00000862   Code   RO          495    .text               os_task.o
    0x00004dda   0x00000002   PAD
    0x00004ddc   0x000001bc   Code   RO          507    .text               os_time.o
    0x00004f98   0x00000574   Code   RO          519    .text               main.o
    0x0000550c   0x00000026   Code   RO          555    .text               lpc11c14_it.o
    0x00005532   0x00000002   PAD
    0x00005534   0x0000003c   Code   RO          570    .text               crc16.o
    0x00005570   0x00000152   Code   RO          584    .text               led_spk_fan_adc.o
    0x000056c2   0x0000002c   Code   RO          601    .text               mc_p.l(uidiv.o)
    0x000056ee   0x00000060   Code   RO          868    .text               mc_p.l(uldiv.o)
    0x0000574e   0x00000002   PAD
    0x00005750   0x00000164   Code   RO          871    .text               mf_p.l(dadd.o)
    0x000058b4   0x000000cc   Code   RO          873    .text               mf_p.l(dmul.o)
    0x00005980   0x000000f0   Code   RO          875    .text               mf_p.l(ddiv.o)
    0x00005a70   0x00000040   Code   RO          877    .text               mf_p.l(dfixul.o)
    0x00005ab0   0x00000028   Code   RO          879    .text               mf_p.l(cdrcmple.o)
    0x00005ad8   0x00000024   Code   RO          881    .text               mc_p.l(init.o)
    0x00005afc   0x00000020   Code   RO          883    .text               mc_p.l(llshl.o)
    0x00005b1c   0x00000022   Code   RO          885    .text               mc_p.l(llushr.o)
    0x00005b3e   0x00000026   Code   RO          887    .text               mc_p.l(llsshr.o)
    0x00005b64   0x000000c4   Code   RO          889    .text               mf_p.l(depilogue.o)
    0x00005c28   0x00000024   Code   RO          841    i.__0vsnprintf      mc_p.l(printfa.o)
    0x00005c4c   0x0000002e   Code   RO          891    i.__ARM_clz         mf_p.l(depilogue.o)
    0x00005c7a   0x0000001c   Code   RO          159    i.__ARM_common_switch8  i2c.o
    0x00005c96   0x0000000e   Code   RO          895    i.__scatterload_copy  mc_p.l(handlers.o)
    0x00005ca4   0x00000002   Code   RO          896    i.__scatterload_null  mc_p.l(handlers.o)
    0x00005ca6   0x0000000e   Code   RO          897    i.__scatterload_zeroinit  mc_p.l(handlers.o)
    0x00005cb4   0x00000154   Code   RO          843    i._fp_digits        mc_p.l(printfa.o)
    0x00005e08   0x0000001e   Code   RO          611    i._printf_core      mc_p.l(printfb.o)
    0x00005e26   0x00000002   PAD
    0x00005e28   0x00000700   Code   RO          844    i._printf_core      mc_p.l(printfa.o)
    0x00006528   0x00000020   Code   RO          845    i._printf_post_padding  mc_p.l(printfa.o)
    0x00006548   0x0000002a   Code   RO          846    i._printf_pre_padding  mc_p.l(printfa.o)
    0x00006572   0x00000016   Code   RO          847    i._snputc           mc_p.l(printfa.o)
    0x00006588   0x00000010   Data   RO           52    .constdata          gpio.o
    0x00006598   0x00000030   Data   RO          257    .constdata          seg7led.o
    0x000065c8   0x00000038   Data   RO          329    .constdata          rfid.o
    0x00006600   0x00000100   Data   RO          396    .constdata          os_core.o
    0x00006700   0x00000200   Data   RO          571    .constdata          crc16.o
    0x00006900   0x00000020   Data   RO          893    Region$$Table       anon$$obj.o


    Execution Region RW_IRAM1 (Base: 0x10000000, Size: 0x00001ed8, Max: 0x00002000, ABSOLUTE)

    Base Addr    Size         Type   Attr      Idx    E Section Name        Object

    0x10000000   0x0000000c   Data   RW           28    .data               system_lpc11xx.o
    0x1000000c   0x0000002c   Data   RW           53    .data               gpio.o
    0x10000038   0x00000010   Data   RW           98    .data               uart.o
    0x10000048   0x00000008   Data   RW          126    .data               retarget.o
    0x10000050   0x00000029   Data   RW          149    .data               i2c.o
    0x10000079   0x00000003   PAD
    0x1000007c   0x00000018   Data   RW          198    .data               ssp.o
    0x10000094   0x00000008   Data   RW          297    .data               light.o
    0x1000009c   0x00000008   Data   RW          352    .data               spi_uart.o
    0x100000a4   0x00000048   Data   RW          397    .data               os_core.o
    0x100000ec   0x0000000c   Data   RW          522    .data               main.o
    0x100000f8   0x00000040   Zero   RW           97    .bss                uart.o
    0x10000138   0x00000020   Zero   RW          177    .bss                adc.o
    0x10000158   0x00000100   Zero   RW          350    .bss                spi_uart.o
    0x10000258   0x0000105c   Zero   RW          395    .bss                os_core.o
    0x100012b4   0x00000b22   Zero   RW          520    .bss                main.o
    0x10001dd6   0x00000002   PAD
    0x10001dd8   0x00000100   Zero   RW            1    STACK               startup_lpc11xx.o


==============================================================================

Image component sizes


      Code (inc. data)   RO Data    RW Data    ZI Data      Debug   Object Name

       386          0          0          0          0       3627   acc.o
       452         28          0          0         32       1892   adc.o
         0          0          0          0          0       4156   core_cm0.o
        60          4        512          0          0       1271   crc16.o
      1256         76         16         44          0      23288   gpio.o
       804         62          0         41          0      17893   i2c.o
       166          0          0          0          0        664   key.o
       338          0          0          0          0       1599   led_spk_fan_adc.o
       752         26          0          8          0       5285   light.o
        38          0          0          0          0       1278   lpc11c14_it.o
      1396        138          0         12       2850       4922   main.o
      3512        316        256         72       4188      20267   os_core.o
       196         40          0          0          0        344   os_cpu_a.o
       300         62          0          0          0      13201   os_cpu_c.o
      2036         46          0          0          0       7304   os_flag.o
      1016         20          0          0          0       4394   os_mbox.o
       436         18          0          0          0       3264   os_mem.o
      1492         32          0          0          0       5797   os_q.o
       952         24          0          0          0       4118   os_sem.o
      2146         70          0          0          0       8037   os_task.o
       444         28          0          0          0       1854   os_time.o
       136         12          0          8          0       3441   retarget.o
       484          4         56          0          0       2473   rfid.o
       144          4         48          0          0       1269   seg7led.o
       720         26          0          8        256       3779   spi_uart.o
       816         44          0         24          0       2858   ssp.o
        32          8        192          0        256       1028   startup_lpc11xx.o
       220         24          0         12          0       8353   system_lpc11xx.o
       532         16          0          0          0       2152   temp_hum.o
       148          8          0          0          0       1135   tools.o
       588         42          0         16         64      11083   uart.o

    ----------------------------------------------------------------------
     22006       1178       1112        248       7648     172026   Object Totals
         0          0         32          0          0          0   (incl. Generated)
         8          0          0          3          2          2   (incl. Padding)

    ----------------------------------------------------------------------

      Code (inc. data)   RO Data    RW Data    ZI Data      Debug   Library Member Name

         0          0          0          0          0          0   entry.o
         8          4          0          0          0          0   entry2.o
         4          0          0          0          0          0   entry5.o
         8          4          0          0          0          0   entry7.o
        30          0          0          0          0          0   handlers.o
        36          8          0          0          0         68   init.o
         0          0          0          0          0          0   iusefp.o
        32          0          0          0          0         68   llshl.o
        38          0          0          0          0         68   llsshr.o
        34          0          0          0          0         68   llushr.o
      2264         96          0          0          0        460   printfa.o
        50          8          0          0          0        144   printfb.o
        44          0          0          0          0         72   uidiv.o
        96          0          0          0          0         84   uldiv.o
        40          2          0          0          0         68   cdrcmple.o
       356          6          0          0          0        140   dadd.o
       240          6          0          0          0         84   ddiv.o
       242          0          0          0          0        216   depilogue.o
        64         10          0          0          0         68   dfixul.o
       204          6          0          0          0         88   dmul.o

    ----------------------------------------------------------------------
      3794        150          0          0          0       1696   Library Totals
         4          0          0          0          0          0   (incl. Padding)

    ----------------------------------------------------------------------

      Code (inc. data)   RO Data    RW Data    ZI Data      Debug   Library Name

      2644        120          0          0          0       1032   mc_p.l
      1146         30          0          0          0        664   mf_p.l

    ----------------------------------------------------------------------
      3794        150          0          0          0       1696   Library Totals

    ----------------------------------------------------------------------

==============================================================================


      Code (inc. data)   RO Data    RW Data    ZI Data      Debug   

     25800       1328       1112        248       7648     170936   Grand Totals
     25800       1328       1112        248       7648     170936   ELF Image Totals
     25800       1328       1112        248          0          0   ROM Totals

==============================================================================

    Total RO  Size (Code + RO Data)                26912 (  26.28kB)
    Total RW  Size (RW Data + ZI Data)              7896 (   7.71kB)
    Total ROM Size (Code + RO Data + RW Data)      27160 (  26.52kB)

==============================================================================

